:1000000000308A0090280000FF00030E8301A10049
:100010007F08A0000A08A8008A01A00E0408A20018
:100020007708A3007808A4007908A5007A08A6003C
:100030007B08A700831383128C308400801D222844
:100040008C193528220884002308F7002408F800BA
:100050002508F9002608FA002708FB0028088A006E
:10006000210E8300FF0E7F0E09008A1143280A101B
:100070008A100A118207023406340E341E343E34CC
:100080007E34FE34FF34290893008C118A11222813
:100090002D308400000803195C280130F800F701B6
:1000A000F70B5028F80B4F284A30F700F70B56286B
:1000B00000000000800B4D280034831605178312C2
:1000C000051F642805136528051783160513831279
:1000D0008A110629AD012D08F93C031C87282C182C
:1000E000732805137428051783160513013083122E
:1000F000AC062C187D2885137E288517831685135A
:100100002130F700F70B82288312AD0A6B28831683
:100110000513831205178316851383128517003480
:1001200084011F30830583161F129F121B0880391C
:100130009B0007309C001C0883120D13603083164F
:100140008F001F129F121B088039D0389B001F138D
:1001500083121F179F1783169F1383121F14941265
:10016000831606118614061200308312940083163B
:1001700094000108C03907388100831290010730CC
:1001800083169C0005080330F700F70BC5281C08F0
:1001900083120D1383169D01861183128611831617
:1001A0000611831206118316861083128610831699
:1001B00085138312851783160513831205172030C4
:1001C000F8001F08C73978049F009501831686112F
:1001D000831286110C3097000030F800043892002A
:1001E00064308316920062308F00023083129500D3
:1001F000AA0183168610831286106430AD00482051
:100200002A08AA0A043C031D07295D28AA018316AF
:100210008610831286140130AD0048201F151F1967
:100220000F291E08503C031CF928831686108312E0
:1002300086106A206430AB00AA012A08073C031C20
:10024000432995010030F800043892002B088316EA
:1002500092001330831295006430AD00482083165D
:100260008610831286140130AD0048201F151F1917
:1002700037291E086A3C0318AB03831686108312C5
:100280008610AA0A1D293830AC00FA30AD0048208B
:10029000AC0B45298316940122308312940002305E
:1002A000A90029089300C0308B0483168C15831293
:1002B000AA012A08073C031C66292A083720F800EF
:1002C000A9003C30AD004820AA0A592983169401A0
:1002D0008312940183168C110611831206150430C3
:1002E000AC00FA30AD004820AC0B71298316061122
:1002F0008312061195016A200830AC00FA30AD0077
:100300004820AC0B7E296A2083160611831206153D
:10031000831685138312851783160513831205131D
:100320000230AC009630AD004820AC0B9229831609
:100330008513831285138316051383120517023064
:10034000AC009630AD004820AC0BA12988291430B0
:10035000AC00FA30AD004820AC0BA9298A01002876
:02036000630038
:04400E003827FC3F14
:00000001FF
